:100000000C948C00189518951895189518951895B6
:100010001895189518951895189518951895189578
:100020001895189518951895189518951895189568
:100030001895189518951895189518951895189558
:100040001895189518951895189518951895189548
:100050001895189518951895189518951895189538
:100060001895189518951895189518951895189528
:100070001895189518951895189518951895189518
:10008000189518951895189518951895392F482F83
:10009000F894E0E0F0E006C001968A352AE0920785
:1000A000D8F33196E017F10718F480E090E0F5CF2F
:1000B0007894842F932F08955A924A92AA939A93F0
:1000C0008A930FEF07BB08BBA1E080E890E04424CF
:1000D000552409C00A2F08BBAA0F04E610E0D6DF9A
:1000E00001E0400E591E08E04016590698F34424DA
:1000F000552408E0401600E0500630F7082F08BBF2
:100100009695879504E610E0C1DF01E0400E591E88
:10011000F0CF00008895FECF0FE30DBF01E00EBFCA
:10012000C0E2D1E00E949A000E945C000E94890017
:080130000C94890001E0089520
:00000001FF
